:020000040000FA
:02000000092ACB
:08000800A000030E8312A10009
:100010002608820020342034203420342034203438
:100020006534733463342E34613473346D34203466
:10003000563431342E3435342034203420342034B6
:100040004534533443344234203420342034203473
:10005000B801B901BA01B90AB601B7010310B50D6B
:10006000B80D03183628B90DBA0D2E28B80CB50CEA
:100070003508B3023808031C013EB402031C4C28A7
:100080003908B6043A08B7040310BA0CB90C0318BF
:100090000800B80CB50C38283508B3070318B40AA3
:1000A0003808B4074428B601B7013508B800381C31
:1000B0005F283308B60734080318013EB70703105A
:1000C000B80C3808031908000310B30DB40D5728F5
:0C00D000313E8200713E8200B13E820091
:1002000085010000062A27088500082200008501D4
:10021000062A2708850005292708850000000B29E4
:10022000270885000E2927088500000012292708C5
:100230008500152927088500000019292708850051
:1002400000001C2927088500042A000085010822D7
:10025000292927088500042A000085010822302961
:100260002729003400340034033409340C341034AA
:10027000133417341A341E34F134F134F134F134B8
:10028000F134F134F134F134F134F134F134F13446
:10029000F134F134F134F134F134F134F134F13436
:1002A000F134F134F134F134F134F134F134F13426
:1002B000F134F134F134F134F134F134F134F13416
:1002C000F134F134F134F134F134F134F134F13406
:1002D000F134F134F134F134F134F1342C34253487
:1002E000223400340034003400340034003400344C
:1002F0000034003400340034FB34FA34F834F7347A
:10030000F534F334F134EF34ED34EB34E934E734DD
:10031000E434E234DF34DC34D934D634D234CF346C
:10032000CB34C734C334BE34B934B434AE34A83457
:10033000A1349A34923489347F34753469345C340E
:100340004D343C3429341334093409340934093424
:1003500009340934093409340934093408340834B7
:100360000834083408340834C834C834C834C834AD
:10037000C834C834C834C834C934C934C934C93499
:10038000C934C934C934C934C934C934C934C93485
:10039000C934C934C934C934C934C934C934C93475
:1003A000C934C934C934C934C934C934C934C93465
:1003B000C934C934C934C934C934C934C934C93455
:1003C000C934C934C934C934CD34D334D934DE3412
:1003D000E434E934EE34F334F834FC3400340034DB
:1003E0000034A218F829A214000085012908FD296B
:1003F000270885002808A210000081000B11210E9B
:100400008300A00E200E09002808FD292908FD29D7
:1004100008008316FF239000831201308A008501B3
:100420008316A83099008312033099008316303068
:1004300002389F001030950000308100DF30FB391A
:10044000FE3985008312FF3081008B16A201143023
:10045000A300A501A701A801A901F130A600FF3062
:10046000AF00B000B100B2008B17EF222218352A7E
:100470004308BC00BE004208BB00403EBD0003185C
:10048000BE0AEF222218412A42083D024308031CFB
:10049000013E3E020318412A4208BD004308BE0047
:1004A0003B083D02B300AD003C08031C013E3E0288
:1004B000B400AE004030B50028203608AC00B300D0
:1004C000B40153203608AD023708031C013EAE02CA
:1004D0000310AE0CAD0C3B08AD073C080318013E01
:1004E000AE07EF222218712A3D0842023E08031C83
:1004F000013E430203184C2A4208B3004308B400EB
:100500001A230038031D712A8B17D522E222D52227
:100510008B17A501A701C5222308A40013232218C5
:100520008C2A6820003C031D8C2AA40B8E2A0130E3
:10053000A300A7018501A501C5222030A700132330
:100540002218892A25020319B12A0318AB2AA50A01
:10055000C52222119F2A221DAF2AA502C5222215DB
:100560009F2A22112608003C031D9F2A851D9F2AD1
:100570000130A7003F30A500C52213232218892A85
:100580006820003C031D992ABD2A25086A20AA007C
:1005900025086C20AB00250868208B12A6002A08CD
:1005A000A8002B08A9008B160800C830BF00203017
:1005B000850008220822082208228501E822BF0BB4
:1005C000D72A0800C830BF00E822BF0BE42A080081
:1005D00064003230C0000822C00BEB2A08002E2332
:1005E000221808000530C1000E08C2000F08C30021
:1005F0002E23221808004208FD3EB3004308031CC6
:10060000FF3EB40033080E02B3003408031C013E61
:100610000F02B400031DEF2A073033020318EF2A3C
:10062000C10BF82A08002E23221800340E08B3004C
:100630000F08B4002D08B3022E08031C013EB402BB
:10064000031C00342C08B5002820B708031D3F34D4
:100650004030360203183F3436080800221040307C
:10066000C4001B30C5008E018F0141309000532320
:10067000221800340E080F040319372B53232218B5
:10068000003409300F0203184D2B051E3E2B90013C
:1006900003300F02031C332B0800532322180034AD
:1006A000051E4D2B332B6400C40B0800C50B08003E
:1006B000221408003108B2003008B1002F08B00041
:1006C0001E08AF00C600C7013008C6070318C70AD6
:1006D0003108C6070318C70A3208C6070318C70A35
:0C06E000C70CC60CC70CC60C460808006E
:02400E00CC3FA5
:00000001FF
